:0200000480007A
:100000006F000005732F2034930F80006308FF03F7
:10001000930F90006304FF03930FB0006300FF038E
:10002000130F000063040F0067000F00732F2034CC
:1000300063540F006F00400093E19153171F0000BD
:1000400023223FFC171F000023200FFC6FF01FFF2F
:100050009300000013010000930100001302000050
:100060009302000013030000930300001304000038
:100070009304000013050000930500001306000020
:100080009306000013070000930700001308000008
:10009000930800001309000093090000130A0000F0
:1000A000930A0000130B0000930B0000130C0000D8
:1000B000930C0000130D0000930D0000130E0000C0
:1000C000930E0000130F0000930F0000732540F102
:1000D0006310050097020000938202017390523072
:1000E000735044749702000093820201739052305F
:1000F00073500018970200009382420273905230AE
:100100009B021000939252039382F2FF7390023B82
:100110009302F0017390023A73504030970200004E
:1001200093824201739052307350203073503030BC
:100130009301000097020000938202ED7390523009
:10014000130510001315F501635C05000F00F00F97
:10015000930110009308D005130500007300000000
:1001600093020000638A020073905210B7B200003D
:100170009B829210739022307350003097020000DF
:100180009382420173901234732540F17300203042
:1001900093012000930000001301000063D62000AB
:1001A0006318303063163000E3DE20FE6312303017
:1001B00093013000930010001301100063D620005B
:1001C0006318302E63163000E3DE20FE6312302EFB
:1001D000930140009300F0FF1301F0FF63D620006D
:1001E0006318302C63163000E3DE20FE6312302CDF
:1001F00093015000930010001301000063D620000B
:100200006318302A63163000E3DE20FE6312302AC2
:1002100093016000930010001301F0FF63D62000EB
:100220006318302863163000E3DE20FE63123028A6
:10023000930170009300F0FF1301E0FF63D62000EC
:100240006318302663163000E3DE20FE631230268A
:1002500093018000930000001301100063D420007C
:100260006314300063163024E3DE20FE9301900017
:100270009300F0FF1301100063D4200063143000DA
:1002800063183022E3DE20FE9301A0009300E0FF1C
:100290001301F0FF63D4200063143000631A302090
:1002A000E3DE20FE9301B0009300E0FF1301100095
:1002B00063D4200063143000631C301EE3DE20FE94
:1002C0009301C000130200009300F0FF130100002F
:1002D00063D0201E1302120093022000E31652FE88
:1002E0009301D000130200009300F0FF13010000FF
:1002F0001300000063DE201A130212009302200094
:10030000E31452FE9301E000130200009300F0FF9B
:1003100013010000130000001300000063DA20182E
:100320001302120093022000E31252FE9301F00028
:10033000130200009300F0FF1300000013010000FF
:1003400063D820161302120093022000E31452FE19
:1003500093010001130200009300F0FF130000005E
:10036000130100001300000063D4201413021200D4
:1003700093022000E31252FE9301100113020000C9
:100380009300F0FF130000001300000013010000B1
:1003900063D020121302120093022000E31252FED7
:1003A00093012001130200009300F0FF13010000ED
:1003B00063D020101302120093022000E31652FEB5
:1003C00093013001130200009300F0FF13010000BD
:1003D0001300000063DE200C1302120093022000C1
:1003E000E31452FE93014001130200009300F0FF5A
:1003F00013010000130000001300000063DA200A5C
:100400001302120093022000E31252FE93015001E6
:10041000130200009300F0FF13000000130100001E
:1004200063D820081302120093022000E31452FE46
:1004300093016001130200009300F0FF130000001D
:10044000130100001300000063D420061302120001
:1004500093022000E31252FE930170011302000088
:100460009300F0FF130000001300000013010000D0
:1004700063D020041302120093022000E31252FE04
:10048000930180019300100063DA00009380100054
:1004900093801000938010009380100093801000D0
:1004A0009380100093033000639470006310300257
:1004B0000F00F00F638001009391110093E1110090
:1004C0009308D00513850100730000000F00F00FA2
:1004D000930110009308D00513050000730000007D
:1004E000731000C0000000000000000000000000C9
:0C04F00000000000000000000000000000
:1010000000000000000000000000000000000000E0
:1010100000000000000000000000000000000000D0
:1010200000000000000000000000000000000000C0
:1010300000000000000000000000000000000000B0
:081040000000000000000000A8
:040000058000000077
:00000001FF
